:10000000000004308A005C2C8030A100FE303121D9
:10001000013031217530A90030307329A101A117B9
:10002000B700B708031D1628030117280130B702CF
:100030000310A30CA30CA30CC0302305403EB7074C
:10004000FE30312137083129A101A117B700FE3058
:10005000312137083129A501B000B101A0112508CF
:100060000319A0150530A4002730AD00103044203E
:100070000330AD00E8304420AD0164304420AD01D0
:100080000A30442030084B28AC003108A900300861
:10009000A80001222808A800A4030319A01125081C
:1000A00003195528240203185C282808031DA011F1
:1000B000A0195C28303E31290800CA00BB1F622805
:1000C0002D303121BD0F6928BC0F6928BB0A0319E7
:1000D000BB0AC201C301C401C501BB176A30BA071C
:1000E0000310BB0CBC0CBD0CC50CC40CC30CC20C67
:1000F000BA0F70283D083A02BD07BA023C083B021D
:10010000BC07BB02A501BC202E303121CB0103105E
:10011000420DBD00430DBC00440DBB00450DBA00AF
:10012000CB0D0310BD0DBC0DBB0DBA0DCB0D4208A0
:10013000BD0743080318430FBC0744080318440FC6
:10014000BB0745080318450FBA070318CB0F031068
:10015000BD0DBC0DBB0DBA0DCB0D4B08303E312192
:100160003D08C2003C08C3003B08C4003A08C50073
:10017000CA0B86280310332AA0112508031DC328A3
:10018000A0150A30A5003D08AB003C08AA003B08BA
:10019000A9003A08A800A401B301B201B1010A30D4
:1001A000B0008721A40A24082502031DCC283008AA
:1001B000031DA011A01DDE28250BE1283008303ECC
:1001C0003121A50BC328332AB500061186118316E9
:1001D000061186110F30860583123508A0180E29E6
:1001E0003E30A900803073213330B4002221133017
:1001F000A9008830732122216430722122216430C9
:1002000072212230B400222128300D210C300D2122
:1002100006300D21A01435080E292014B400201C2E
:100220001C298611033C031C212921210730A90028
:10023000D0307321031408002014FE3C03192F2929
:100240008615201C201006150F3086053408F0395D
:1002500086040611B40E2018222932307221350886
:10026000332AA11BE4280800A400A20124080317D4
:100270008D000313250803178F0047210319332A24
:100280003121A40A0319A50AA20F3629332A83169D
:1002900003178C170C140000000083120C08332A7B
:1002A000B400B40DB40D340D3839C1389F00B41A00
:1002B0009F14323072211F151F195C291E08BB00C4
:1002C00083161E088312BA00332AAD01AC00FF303A
:1002D000AC07031CAD07031C332A0330A900DF3031
:1002E00073216729A901E83EA800A909FC30031C75
:1002F0007C29A80703187929A8070000A90F7929E4
:1003000028188229A81C86290000862908002B08A5
:1003100033068039B500AB1F9829A809A909AA0995
:10032000AB09A80A0319A90A0319AA0A0319AB0AF7
:10033000B31FA529B009B109B209B309B00A03195D
:10034000B10A0319B20A0319B30AAC01AD01AE0137
:10035000AF01BE01BF01C001C10133083204310445
:1003600030040319E3292030B4000310A80DA90DAF
:10037000AA0DAB0DBE0DBF0DC00DC10D330841025E
:10038000031DCC2932084002031DCC2931083F024D
:10039000031DCC2930083E02031CDD293008BE02B3
:1003A0003108031C310FBF023208031C320FC00298
:1003B0003308031C330FC1020314AC0DAD0DAE0D99
:1003C000AF0DB40BB529B51FF029AC09AD09AE09C5
:1003D000AF09AC0A0319AD0A0319AE0A0319AF0A33
:1003E0003E08B0003F08B1004008B2004108B30029
:1003F0002C08A8002D08A9002E08AA002F08AB0081
:10040000332AB101B0011030B400290DB00DB10D87
:100410002C08B0022D08031C2D0FB1020318172A57
:100420002C08B0072D0803182D0FB1070310A80DD5
:10043000A90DB40B052A2808332A1030B900A901E8
:10044000A801B50CB40C031C2B2A2C08A8072D08F6
:1004500003182D0FA907A90CA80CB10CB00CB90BEF
:10046000212A3008332A8313831203130800470814
:100470004306CE00CE1B6C2AC71B552A46084202F3
:10048000031C0034031D013447084302031C0034DD
:10049000031D013448084402031C0034031D0134C9
:1004A00049084502031C0034013442084602031C7B
:1004B0000034031D013443084702031C0034031DAC
:1004C000013444084802031C0034031D013445086C
:1004D0004902031C00340134C31F013400344608B0
:1004E0004202CA0003188E2ACA09CA0A4208CD006D
:1004F0004608C2004D08C6004308CD004708C300A7
:100500004D08C7004408CD004808C4004D08C80085
:100510004508CD004908C5004D08C9001A304A02F7
:100520000318332AC6080319332ABE014308CD0035
:100530004706CF00C317C7170830CA02031CA82AF2
:100540004908BE004808C9004708C800C7019C2ADE
:10055000CA070319B42A0310C70CC80CC90CBE0C77
:10056000CA03CA08031DAB2ACF1FFD2A4908C502CA
:100570004808031C480FC4024708031C470FC30266
:100580000318CC2AC309C409C509C50FCA2AC40A5D
:100590000319C30A8030CD06BE09BE0A0319D72A43
:1005A000C503450FD72AC403440A0319C303043003
:1005B000CA00C308031DEB2A4408C3004508C40051
:1005C0003E08C500BE010830C202031C1E2BCA0330
:1005D00003191E2BD92AC31BF62A0310BE0DC50D05
:1005E000C40DC30DC20303191E2BEB2A4C1FFC2A9A
:1005F000BE1FFC2ABE01142B1D2B4908C507480845
:100600000318480FC40747080318470FC307031C04
:10061000102BC30CC40CC50CBE0CC20A0319202B32
:100620004C1F1D2BBE1F1D2BC50F1D2BC40F1D2BBB
:10063000C30F1D2B03144210092B272BC201232BA0
:10064000CC16FF30C200C501C4018030C300CD1BF1
:100650002A2BC313332A4308C0004706CF00C6081D
:100660000319952BC2080319982B4608C2027F3044
:1006700003183E2BC207031C972B412BC2070318FC
:100680009A2B4508BE004408BF00C017C717183092
:10069000CD00C501C401C3014F2B03185B2B4908D2
:1006A0003E024808031C480F3F024708031C470F3F
:1006B0004002031C662B4908BE024808031C480F71
:1006C000BF024708031C470FC0020314C50DC40D29
:1006D000C30DBE0DBF0DC00DCD0B4D2BC31B782B15
:1006E000C2080319972BCF0CC203CD0ACF0D4D2B97
:1006F0004C1F942B0318882B4908BE024808031C82
:10070000480FBF024708031C470FC002031C942B6D
:10071000C50F942BC40F942BC30F942BC30CC40C84
:10072000C50CC20A03199A2BA12BCC159B2B4C1577
:10073000C2019D2BCC14FF30C200C501C401803022
:10074000C300CF1BA42BC313332A4308C0004706A2
:10075000CF004208003A031D4608003A0319F72B60
:10076000C2077E30031CB82BC2020318F92BBB2B27
:10077000C202031CF62B4508BE004408BF00C01788
:10078000C717C501C401C3011830CD00C00CBF0C90
:10079000BE0C031CD52B4908C50748080318480F91
:1007A000C40747080318470FC307C30CC40CC50C84
:1007B000CD0BC62BC31BE42BC50DC40DC30DC20846
:1007C0000319F62BC203400D4C1FF52B031CF52B10
:1007D000C50FF52BC40FF52BC30FF52B0314C30C5A
:1007E000C40CC50CC20A0319F92B002C4C15C2010C
:1007F000FC2BCC14FF30C200C501C4018030C30003
:10080000CF1B032CC313332AC401C5019630CD007E
:10081000CF13C51F172CC509C409C309C209C20FCC
:10082000162CC30F162CC40A0319C50ACF17C50806
:100830000319322C4C1F292CC51F292CC30F292C1E
:10084000C40F292CC50F292C0314C50CC40CC30CD0
:10085000CD0A0830CD074308C2004408C30045084C
:10086000C400472CC408031D472C0830CD024308A0
:10087000031D432C0830CD024208031D422C4508BD
:10088000CD00512CC201C4004208C300C201C41BE8
:100890004F2C0310C20DC30DC40DCD03472CCF1F29
:1008A000C4134208C5004D08C2004408CD004308E7
:1008B000C4004D08C300332A4030CC00A0010730EB
:1008C00083169F00FF30850086018701880107306D
:1008D000890082309F008312D0010A30EF00F001BE
:1008E000F501F401F301F201F101F901F801F70159
:1008F000F601FD01FC01FB01FA012D30D500FE30AF
:100900008A01E42040308A01E4200E308A01E4208C
:1009100011308A01E42010308A01E42010308A016D
:10092000E42010308A01E42015308A01E4200E30E2
:100930008A01E42000308A01E420FE308A01E420AC
:1009400048308A01E4200E308A01E42011308A0107
:10095000E42011308A01E42011308A01E4201130B2
:100960008A01E42011308A01E4201F308A01E4204A
:1009700000308A01E420FE308A01E42050308A01F0
:10098000E4200E308A01E42011308A01E420113085
:100990008A01E42011308A01E4201F308A01E4201A
:1009A0001F308A01E4201F308A01E42000308A01D0
:1009B000E420FE308A01E42058308A01E42004302B
:1009C0008A01E4200E308A01E42004308A01E42008
:1009D00004308A01E42004308A01E42004308A01D2
:1009E000E4200E308A01E42000308A01E420FE3049
:1009F0008A01E42060308A01E4200E308A01E4207C
:100A000011308A01E42010308A01E4200E308A017E
:100A1000E42001308A01E42015308A01E4200E3000
:100A20008A01E42000308A01E420FE308A01E420BB
:100A300068308A01E4200E308A01E42000308A0107
:100A4000E4200F308A01E42010308A01E4201730BE
:100A50008A01E42011308A01E4200F308A01E42069
:100A600000308A01E420FE308A01E42070308A01DF
:100A7000E4200E308A01E42011308A01E4201F3086
:100A80008A01E4201F308A01E4201F308A01E4201B
:100A90001F308A01E4201F308A01E42000308A01DF
:100AA000E420FE308A01E42078308A01E4200E3010
:100AB0008A01E4201F308A01E4201F308A01E420EB
:100AC0001F308A01E4201F308A01E4201F308A0190
:100AD000E4201F308A01E42000308A01E420003045
:100AE000870088000130AD00F4308A0166218A1544
:100AF0000A121D248030A1008A01242050308A016E
:100B0000E42003308A01E4200F30A500AB308A01D5
:100B1000342103308A01E4204E308A01E42003307E
:100B20008A01E42020308A01E4208A01E4208A013D
:100B3000E4208A01E4208A01E4208030A100C03052
:100B40008A01242047308A01E42003308A01E4200E
:100B500052308A01E42003308A01E4200F30A500DE
:100B6000B2308A0134210330AD00E8308A016621B9
:100B70008A110A128918BF2D8A110A12C8258A11F2
:100B80000A120919C62D8A110A12312E8A01B82DAE
:100B9000FA308A016521D00A0D3050028A110A12FA
:100BA000031CD42D0130D000D0088A110A12031D75
:100BB000DB2D8A01C82D8A0104208030A1008A0122
:100BC000242050088A012B2083308A0124205030B1
:100BD0008A01E42003308A01E4204C308A01E420B9
:100BE0002A308A01E42027308A01E42042308A0139
:100BF000E42041308A01E42004308A01E4204C30B2
:100C00008A01E42041308A01E42027308A01E4206F
:100C100059308A01E42041308A01E4208030A1006B
:100C2000C0308A0124200F30A500BF308A01342152
:100C300000308A01E42041308A01E4204C308A01EE
:100C4000E42049308A01E42004308A01E420543051
:100C50008A01E42049308A01E42052308A01E420EC
:100C60000800D0088A110A12031D392E8A150A12AB
:100C7000642D5008B400B5011330AC00AD018A01F9
:100C80001D22EA003108EB006A08C2006B08C300AD
:100C90008A010424C901C8012030C7008330C6007E
:100CA0008A016F224508BD004408BC004308BB0010
:100CB0004208BA00C901C8012030C7008230C6000E
:100CC0003D08C5003C08C4003B08C3003A08C20008
:100CD0008A012B234508E9004408E8004308E7009F
:100CE0004208E600EC01ED01EE0103308A015021DB
:100CF000A6003B08A7002608EC0727080318013EBA
:100D0000ED07EE0A6E086F028A110A12031D752E96
:100D10006C08A8006D08A9006F08AC00AD018A013D
:100D20000122EC002908ED006C08C2006D08C30028
:100D30008A0104244508E5004408E4004308E30070
:100D40004208E200C501C401C3017F30C20065084A
:100D5000C9006408C8006308C7006208C6008A01A9
:100D60006F224508E5004408E4004308E300420818
:100D7000E200C501C4014830C3008430C2006508E8
:100D8000C9006408C8006308C7006208C6008A0179
:100D9000A5234508BD004408BC004308BB00420829
:100DA000BA003D08E5003C08E4003B08E3000A30D7
:100DB0003A028A110A120318DF2E4C150030E200A5
:100DC0001E308A0165216508C5006408C4006308F7
:100DD000C3006208C2006908C9006808C800670843
:100DE000C7006608C6008A013722013C8A110A1230
:100DF0000319FD2E8A150A123D29013050028A116D
:100E00000A12031D052F11308700023050028A118B
:100E10000A12031D0D2F21308700033050028A1162
:100E20000A12031D152F41308700043050028A1129
:100E30000A12031D1D2F81308700053050028A11D0
:100E40000A12031D252F12308700063050028A1126
:100E50000A12031D2D2F22308700073050028A11FD
:100E60000A12031D352F42308700083050028A11C4
:100E70000A12031D3D2F82308700093050028A116B
:100E80000A12031D452F143087000A3050028A11C0
:100E90000A12031D4D2F243087000B3050028A1197
:100EA0000A12031D552F443087000C3050028A115E
:100EB0000A12031D5D2F843087008A0104208030D0
:100EC000A1008A0124200F30A500C8308A013421F6
:100ED00004308A01E4204C308A01E42041308A0148
:100EE000E42044308A01E42049308A01E4202130A2
:100EF0008A01E4200130D300063053028A110A121D
:100F00000318AB2F0130D200123052028A110A129C
:100F10000318A62F8030A1000230A30052088A01D6
:100F200010203E308A01E4208030A1000230A3006E
:100F300052038A01102020308A01E42032308A01D5
:100F40006521D20A8A110A12031D842FD30A8A113D
:100F50000A12031D7C2F8A0104208030A1008A011F
:100F6000242027308A01E42042308A01E4204130E5
:100F70008A01E42004308A01E4204C308A01E42014
:100F800041308A01E4202F308A01E42042308A0176
:100F9000E42003308A01E42054308A01E420033045
:100FA0008A01E4200F30A500D4308A0134210530B5
:100FB000AD00DC308A0166218030A1008A01242046
:100FC00027308A01E42042308A01E42003308A017C
:100FD000E42054308A01E42003308A01E4205230B6
:100FE0008A01E42027308A01E4204C308A01E42081
:100FF00045308A01E42020308A01E42003308A0150
:10100000E42050308A01E42054308A01E420413049
:101010008A01E4204C308A01E4208030A100C030F5
:101020008A01242045308A01E42044308A01E420EA
:1010300045308A01E42042308A01E42003308A01ED
:10104000E4204C308A01E42003308A01E42052304D
:101050008A01E42053308A01E42003308A01E4202D
:101060004E308A01E42003308A01E4205A308A019C
:10107000E4202E308A01E4200B30AD00B8308A0124
:1010800066218A0104208A150A1209194A288A153C
:101090000A12E02A8A150A12891851288A150A129A
:1010A000B325FA308A0165218A150A12BF208A15F4
:1010B0000A1243288A0104208030A1008A012420DA
:1010C0002A308A01E42020308A01E42050308A014D
:1010D000E42003308A01E4200F30A500DD308A01CE
:1010E00034218030A100C0308A0124200F30A500B7
:1010F000EB308A01342103308A01E4200F30A5004F
:10110000F2308A0134210B30AD00B8308A016621FB
:101110008030A1008A0124200F30A500FC308A0114
:10112000342103308A01E4201030A50003308A0105
:1011300034218030A100C0308A01242050308A013F
:10114000E42003308A01E4204C308A01E4208A0143
:10115000E42045308A01E42052308A01E420033043
:101160008A01E4201030A5000D308A0134210B30B3
:10117000AD00B8308A0166218A150A125A288030DB
:10118000A1008A01242050088A012B2083308A0183
:10119000242020308A01E42050308A01E4200330EA
:1011A0008A01E4204C308A01E4203E308A01E420A8
:1011B0008030A1008F308A01242001308A01E42090
:1011C000023050028A150A12031CEE288030A1005A
:1011D0008E308A01242001308A01E42064308A01A3
:1011E00065218030A1008F308A01242002308A01DD
:1011F000E420023050028A150A12031C07298030AD
:10120000A1008E308A01242002308A01E42064305B
:101210008A0165218030A1008F308A0124200630A8
:101220008A01E420023050028A150A12031C202988
:101230008030A1008E308A01242006308A01E4200B
:1012400064308A0165218030A1008F308A0124201A
:1012500007308A01E420023050028A150A12031C6A
:1012600039298030A1008E308A01242007308A017C
:10127000E42064308A016521080088140130AD0043
:101280002C308A016621F00A023070028A150A1297
:10129000031C4D298A150A124F298A01FD2E8A0145
:1012A00004200130D100043051028A150A120318BB
:1012B00071298030A1001030A50017308A01342137
:1012C0000130AD00F4308A0166218A01042001302A
:1012D000AD00F4308A016621D10A8A150A12031D75
:1012E00053298030A1008A0124201030A500273026
:1012F0008A01342103308A01E4204E308A01E4203F
:1013000020308A01E4208030A100C0308A012420EE
:1013100000308A01E42041308A01E4204C308A0107
:10132000E42049308A01E42004308A01E42041307D
:101330008A01E42042308A01E42003308A01E4205B
:101340004C308A01E4204D308A01E42045308A0186
:10135000E42053308A01E42003308A01E42007307E
:10136000AD00D0308A0166218A0104208030A100BE
:101370008A0124201030A50031308A013421033045
:101380008A01E4204C308A01E42029308A01E420DB
:1013900056308A01E4208030A100C0308A01242028
:1013A00004308A01E4201030A5003A308A0134214B
:1013B00005308A01E4201030A50044308A01342130
:1013C0000B30AD00B8308A0166218A0104208030DC
:1013D000A1008A01242050088A012B201030A5008A
:1013E0004B308A01342103308A01E4204C308A01D9
:1013F000E42020308A01E42003308A01E420003018
:101400008A01E42003308A01E4204E308A01E4207E
:101410008030A100C0308A0124204D308A01E420B0
:1014200003308A01E4204E308A01E4202E308A0104
:10143000E4206908BD006808BC006708BB006608B6
:10144000BA0001308A015D201030A50053308A01B6
:10145000342103308A01E4200B30AD00B8308A011A
:1014600066218A0104208030A1008A0124200430F2
:101470008A01E4201030A5005D308A0134218030DB
:10148000A100C0308A01242047308A01E420453081
:101490008A01E42052308A01E42003308A01E420EA
:1014A0004C308A01E42003308A01E4204D308A0167
:1014B000E42003308A01E42020308A01E42065081A
:1014C000BD006408BC006308BB006208BA000130BC
:1014D0008A015D2020308A01E42056308A01E42010
:1014E00021308A01E4200730AD00D0308A01662126
:1014F0008A0104208030A1008A01242047308A011B
:10150000E42045308A01E42052308A01E42003308F
:101510008A01E4204C308A01E42003308A01E4206F
:101520004D308A01E4208030A100C0308A0124209F
:101530001030A5006D308A01342103308A01E42087
:101540005A308A01E42021308A01E4200730AD00BE
:10155000D0308A0166218A0104208030A1008A01EE
:1015600024201030A50074308A01342103308A0110
:10157000E4204C308A01E42003308A01E4202D303D
:101580008A01E4208030A100C0308A0124204D303F
:101590008A01E42003308A01E4204E308A01E420ED
:1015A00003308A01E4201030A50080308A01342104
:1015B0000B30AD00B8308A0166218A150A125C2B07
:1015C0000030870088008A0104208A0104208030CE
:1015D000A1008A0124201030A5008A308A0134211C
:1015E00003308A01E42050308A01E42054308A011B
:1015F000E42041308A01E4204C308A01E42080302C
:10160000A100C0308A01242045308A01E4205430F2
:101610008A01E42044308A01E42003308A01E42076
:101620004E308A01E42003308A01E4205A308A01D6
:10163000E4200730AD00D0308A0166218030A1005F
:101640008A0124201030A50096308A01342103300D
:101650008A01E4201030A5009D308A0134218030B9
:10166000A100C0308A01242050308A01E4200330D8
:101670008A01E4204C308A01E4208A01E4204530CC
:101680008A01E42052308A01E42003308A01E420F8
:101690001030A500A8308A0134210730AD00D030C9
:1016A0008A01662188150130AD00F4308A01662177
:1016B00088118A150A12E52A0030870088008A01FD
:1016C00004208030A1008A01242047308A01E420D0
:1016D00045308A01E42052308A01E42003308A0137
:1016E000E4204C308A01E42003308A01E4204D30AC
:1016F0008A01E4208030A100C0308A01242010300B
:10170000A500B2308A01342103308A01E4205A3026
:101710008A01E4204C308A01E42003308A01E4206D
:1017200005308A01E42003308A01E4204E308A012A
:10173000E42044308A01E42045308A01E4204E3020
:101740008A01E4200730AD00D0308A016621803064
:10175000A1008A0124201030A500B9308A0134216B
:1017600003308A01E4201030A500C3308A013421FF
:101770008030A100C0308A01242045308A01E42055
:1017800044308A01E42003308A01E4204C308A018D
:10179000E42044308A01E42003308A01E420103040
:1017A000A500CA308A0134210730AD00D0308A014B
:1017B00066218030A1008A0124201030A500D53098
:1017C0008A01342103308A01E4201030A500DC3086
:1017D0008A0134218030A100C0308A012420503099
:1017E0008A01E42003308A01E4204C308A01E4209D
:1017F0008A01E42045308A01E42052308A01E42045
:1018000003308A01E42020308A01E42000308A017C
:10181000E4201030A500E6308A0134210730AD0005
:10182000D0308A01662188150130AD00F4308A017C
:10183000662188118A150A125F2B8A010420103054
:10184000D400023054028A150A12031C442C803042
:10185000A1000130A30054088A0110202A308A0117
:10186000E4208030A1000130A300540A8A01102036
:1018700020308A01E42055088A0165210130D40214
:101880008A150A120318212C1030D4000430540297
:101890008A150A12031C692C8030A1000130A300B4
:1018A00054088A01102054308A01E4208030A100BD
:1018B0000130A300540A8A01102020308A01E4205C
:1018C00055088A0165210130D4028A150A120318CD
:1018D000462C1030D400063054028A150A12031C1C
:1018E0008E2C8030A1000130A30054088A01102002
:1018F00041308A01E4208030A1000130A300540A65
:101900008A01102020308A01E42055088A016521CF
:101910000130D4028A150A1203186B2C1030D4003F
:10192000083054028A150A12031CB32C8030A1001F
:101930000130A30054088A01102032308A01E420CB
:101940008030A1000130A300540A8A011020203009
:101950008A01E42055088A0165210130D4028A15E4
:101960000A120318902C1030D4000A3054028A1541
:101970000A12031CD82C8030A1000130A3005408A7
:101980008A01102045308A01E4208030A100013016
:10199000A300540A8A01102020308A01E42055084F
:1019A0008A0165210130D4028A150A120318B52C68
:1019B0001030D4000C3054028A150A12031CFD2C7E
:1019C0008030A1000130A30054088A011020493062
:1019D0008A01E4208030A1000130A300540A8A016A
:1019E000102020308A01E42055088A016521013049
:1019F000D4028A150A120318DA2C1030D4000E30E3
:101A000054028A150A12031C222D8030A1000130D5
:101A1000A30054088A0110202A308A01E420803073
:101A2000A1000130A300540A8A01102020308A014D
:101A3000E42055088A0165210130D4028A150A1272
:101A40000318FF2C8030A1008E308A012420203022
:101A50008A01E4208A01E4200330AD0020308A01AD
:101A600066210130D400043054028A150A1203188A
:101A7000542D8A0104200130AD00F4308A01662122
:101A80008030A10081308A0124201030A500EE3082
:101A90008A0134210330AD0020308A016621D40A46
:101AA0008A150A12031D332D8030A100C0308A012F
:101AB00024201030A500FC308A0134210F30AD0005
:101AC000A0308A01662108008030A1008A0124200C
:101AD00050308A01E42003308A01E4201130A5004F
:101AE0000D308A01342103308A01E4204E308A010E
:101AF000E42003308A01E42020308A01E4208A01B6
:101B0000E4208A01E4208A01E4208A01E420803074
:101B1000A100C0308A01242047308A01E42003302C
:101B20008A01E42052308A01E4204D308A01E42009
:101B300045308A01E42044308A01E42003308A01E0
:101B4000E4204E308A01E42003308A01E420113081
:101B5000A50014308A0134210B30AD00B8308A0161
:101B600066218A017A2DD3018030A1008A012420C8
:101B70001130A5001C308A0134218030A100C03012
:101B80008A0124201130A5002D308A01342107302C
:101B9000AD00D0308A0166218030A1008A01242066
:101BA00004308A01E4201130A5003E308A0134213E
:101BB0008030A100C0308A01242042308A01E42014
:101BC00041308A01E42004308A01E4204C308A014B
:101BD000E42041308A01E4202F308A01E4204230A1
:101BE0008A01E42003308A01E42054308A01E42091
:101BF00003308A01E42052308A01E42020308A0137
:101C0000E42054308A01E42055308A01E420043075
:101C10008A01E42055308A01E4200230AD00BC3056
:101C20008A0166218030A1008A01242042308A0185
:101C3000E42041308A01E42004308A01E4204C3061
:101C40008A01E42041308A01E4202F308A01E42017
:101C500042308A01E42003308A01E42054308A01B2
:101C6000E42003308A01E42052308A01E42020304D
:101C70008A01E42054308A01E42055308A01E420AE
:101C800004308A01E42055308A01E4208030A1002C
:101C9000C0308A01242003308A01E4204C308A01BC
:101CA000E42045308A01E42020308A01E420043019
:101CB0008A01E42041308A01E42052308A01E42084
:101CC0004A308A01E42049308A01E42020308A0128
:101CD000E42003308A01E4201130A5004E308A014F
:101CE00034210230AD00BC308A0166218030A10071
:101CF0008A01242003308A01E4204C308A01E42048
:101D000045308A01E42020308A01E42004308A0131
:101D1000E42041308A01E42052308A01E4204A3034
:101D20008A01E42049308A01E42020308A01E4203D
:101D300003308A01E4201130A50055308A01342196
:101D40008030A100C0308A01242045308A01E4207F
:101D500044308A01E42045308A01E42042308A017F
:101D6000E42003308A01E4204C308A01E42003306F
:101D70008A01E42052308A01E42053308A01E420B1
:101D800003308A01E4204E308A01E42003308A01C6
:101D9000E4205A308A01E4202E308A01E4202030E9
:101DA0008A01E4208A01E4200730AD00D0308A01A6
:101DB00066218030A1008A0124201130A5005C300A
:101DC0008A01342103308A01E4201130A5006630F5
:101DD0008A0134218030A100C0308A0124200030E3
:101DE0008A01E42041308A01E4204C308A01E42059
:101DF00049308A01E42004308A01E42041308A011C
:101E0000E42042308A01E42003308A01E4204C308F
:101E10008A01E4204D308A01E42045308A01E42023
:101E200053308A01E42003308A01E42020308A0103
:101E3000E4208A01E4208A01E4208A01E4200230BF
:101E4000AD00BC308A0166218030A1008A012420C7
:101E500000308A01E42041308A01E4204C308A01BC
:101E6000E42049308A01E42004308A01E420413032
:101E70008A01E42042308A01E42003308A01E42010
:101E80004C308A01E4204D308A01E42045308A013B
:101E9000E42053308A01E42003308A01E42020301A
:101EA0008A01E4208A01E4208A01E4208A01E420F6
:101EB0008030A100C0308A0124201130A5006D308F
:101EC0008A01342103308A01E4201130A5007630E4
:101ED0008A0134210230AD00BC308A016621803095
:101EE000A1008A0124201130A5007E308A0134210E
:101EF00003308A01E4201130A50087308A013421A3
:101F00008030A100C0308A01242004308A01E420FE
:101F10001130A5008F308A01342105308A01E42078
:101F20001130A50099308A0134210F30AD00A03066
:101F30008A016621D30A033053028A150A12031C50
:101F4000B42D8A010420080063008A150A12A42F08
:101F50008A150A12A82F4C002000410044004500B9
:101F6000440000004E002E002E0020002000200023
:101F7000200020002000200020002000000042005F
:101F8000410053004100520041004B00200000007E
:101F900044004F004C004400550052004D004100E9
:101FA0002000420041000000520027004C00450084
:101FB000200020002000200000004C004C004500C4
:101FC0005200200044004F004C00440055002C00FB
:101FD000200020000000440045005600520045004B
:101FE0005900000020004B00410050004100540007
:101FF00049005000200000004400450056005200F7
:1020000045005900000020004B00410050004100F5
:102010005400490050002000000020004300490007
:102020004B0041005200540049004E0000002A00BD
:102030002A002A002000440069004B004B004100A8
:102040005400210020002A002A002A00000042003B
:1020500055002000440045005600520045004E0047
:10206000000032002B00280031002C0039002A002B
:102070005000000041005200540049004E00410051
:1020800020004200410000004C004900440049008B
:10209000520021000000200041004400450054008F
:1020A000200050000000200056002000470045009E
:1020B000520045004B004C0000005500200041003C
:1020C0004E004400410020004200450053004C00F7
:1020D00045004D0045002000000059004500540017
:1020E00045005200530000004200450053004C00E0
:1020F00045004D004500200047004500520000000B
:102100002000410052005400540049005200490090
:102110004E00000044004F004C00440055005200A7
:102120004D004100590049002000000044004500D6
:102130005600520045005900000020004B004100AD
:1021400050004100540049004E002C0020000000C7
:102150002000430049004B00410052005400490058
:102160004E00000059004500540045005200530045
:10217000000044004F004C004400550052004D0048
:102180004100200000005000540041004C0020009D
:10219000200000002000200020002000200020005F
:1021A00020002000200020000000440045005600D0
:1021B000520045005900000020004B004100500033
:1021C0004100540049004E002C00000049004B0023
:1021D00041005200540049004E0000002A00200037
:1021E0005400200041002000320020004500200063
:1021F000490020002A0000004D004100580037002F
:1022000031003300200044004F004C0044005500D2
:10221000520055004300550000004C0020004100D2
:1022200044004500440000005A0020002000200027
:10223000200020002000000044004F004C0044001B
:10224000550052004D00410020005A0041004D0051
:1022500041004E004900200000004D0041005800A0
:102260002E00320036003400200044004B002E00C7
:102270004B00410044004900520000004100520060
:102280004A002000590041005000410052004B001C
:1022900045004E00200020002000000050005400A7
:1022A00041004C002000200000005000540041007C
:1022B0004C00200020000000420055002000440097
:1022C00045005600520045004E0000004E00200020
:1022D0002000200020002000000032002B002800F9
:1022E00031002C0039002A00500000004C00290069
:1022F00056002000200020002000000032002B00AB
:10230000280031002C0039002A00500000004C0049
:10231000290056002000200020002000000041007D
:102320005200540049004E0041002000420041008C
:1023300000004C0049004400490052002100000008
:02400E00323F3F
:00000001FF
